:020000040000FA
:06000000EAEF18F0120007
:06080000EAEF18F01200FF
:06080800F5EF07F01200FD
:06082A0001004432000051
:08083000600000004800000018
:08083800D9CFE6FFE1CFD9FFA3
:10084000040EE126DE6ADE6ADE6ADD6ADD52DD5212
:10085000FD0EDBCF14F0FE0EDBCF15F0166A176A23
:1008600015AE02D016681768D9CFE9FFDACFEAFFD4
:10087000030EEB501718E8AE02D0173408D014500E
:10088000EE5C1550EE581650EE581750EE580FE229
:100890000C0EE66ECAEC18F0E552D9CFE9FFDACFBC
:1008A000EAFFEE2A000EEE22EE22EE22D1D7040E4F
:1008B000E15C02E2E16AE552E16EE552E7CFD9FF81
:1008C00012000F0EC16E070EB46E936A300E926E58
:1008D0000F0E946EF19E1200D9CFE6FFE1CFD9FF43
:1008E000020EE1268250020B01E0010E080DF3CF4B
:1008F00016F08250010B040DF3CF15F08050200B41
:1009000001E0010EE824146E8050100B01E0010E8E
:10091000142415241624DE6EDD6ADECF14F0DDCF3C
:1009200015F014C0F3FF15C0F4FF020EE15C03E202
:1009300000D0E16AE552E16EE552E7CFD9FF12003F
:100940008092320EE66E06EC19F0E5528084320E8B
:10095000E66E06EC19F0E5528094320EE66E06EC77
:1009600019F0E55212008082320EE66E06EC19F0A4
:10097000E5528084320EE66E06EC19F0E552809462
:10098000320EE66E06EC19F0E5521200380E816E5A
:10099000D7DF320EE66EE66A4FDFE552E552010E12
:1009A000816ECEDF320EE66EE66A46DFE552E55234
:1009B0000D0E816EC5DF320EE66EE66A3DDFE55252
:1009C000E552060E816EBCDF320EE66EE66A34DF5B
:1009D000E552E5521200010E816EB2DF0A0EE66E9C
:1009E000E66A2ADFE552E5521200D9CFE6FFE1CFF1
:1009F000D9FF020E816EA4DF0A0EE66EE66A1CDFE6
:100A0000E552E552FD0EDBCFE6FFFE0EDB50280D72
:100A1000F350E552E724E76EFE0EE7CFDBFFFD0E55
:100A2000DB6AFE0EDB50F36EFD0EDBCFF4FFF350FE
:100A3000F45C0BE2140E816E83DF320EE66E06EC80
:100A400019F0E552FD0EDB2AECD7E552E7CFD9FFCE
:100A50001200D9CFE6FFE1CFD9FFFE0EDB50816E49
:100A600082DF320EE66E06EC19F0E552E552E7CF72
:100A7000D9FF1200D9CFE6FFE1CFD9FFFD0EDBCFC2
:100A8000E9FFFE0EDBCFEAFFEF500EE0FD0EDBCFFD
:100A9000E9FFDB2AFE0EDBCFEAFF01E3DB2AEF50A2
:100AA000E66ED7DFE552EAD7E552E7CFD9FF12006D
:100AB0000201046B300E926EF00E936EEF0E006F1B
:100AC00000C281FF040E016F0151000821E20051B4
:100AD000FE0BE842006F00C281FF050EE66EE66A7B
:100AE000ABDEE552E5528150100B09E08150200B3E
:100AF00006E08150400B03E08150800B01E10AD8F1
:100B00000201040502E1055104D00105016FDCD7A3
:100B1000CFD71200F00E936E81CF03F202010315BE
:100B2000026F0F0E0015006F00510211006F81CF90
:100B300003F2F00E0315026FF00E025D01E0F7D72D
:100B4000936A06D806C205F20201010E046F120074
:100B50000201076B100E075D14E20751EA6A600F8D
:100B6000E96E000EEA22EF50005D08E10751EA6AE3
:100B7000700FE96E000EEA22EFCF06F20729076F29
:100B8000E9D706C281FF640EE66EE66A55DEE552DD
:100B9000E55212000201086B070E085D1DE288DFB6
:100BA0000201096F0851EA6A0A0FE96E020EEA2291
:100BB00009C2EFFF0851EA6A0A0FE96E020EEA2243
:100BC000EF50460802E108D004D009C2E6FF41DF39
:100BD000E5520201082BE0D70851EA6A0A0FE96ED4
:100BE000020EEA22EF6A12000201086B070E085D8E
:100BF00016E20851EA6A0A0FE96E020EEA22EF5085
:100C0000E66E27DFE55202010829EA6A0A0FE96E5B
:100C1000020EEA22EF5001E102D0082BE7D71200C2
:100C2000D9CFE6FFE1CFD9FFE652F250800B01E0C9
:100C3000010EDF6EF29EA69EA69CA684FE0EDB50E1
:100C4000A96EFD0EDB50A86E550EA76EAA0EA76EFC
:100C5000A682A6B2FED7A694DF50E8B0F28EE8A036
:100C6000F29EE552E552E7CFD9FF1200D9CFE6FF59
:100C7000E1CFD9FFA69CA69EFE0EDB50A96EA680F2
:100C8000A85000D0E552E7CFD9FF1200D9CFE6FF38
:100C9000E1CFD9FF0E0EE126DE6ADD6AB6D8CC0EB2
:100CA000E66EE66AC3D8E552E552440EE66EE66AA1
:100CB000BDD8E552E552D9CFE9FFDACFEAFFEE50D1
:100CC000ED1006E11ED9F3CFDEFFF4CFDDFFF3D741
:100CD0009CD8CC0EE66EE66AA9D8E552E552BE0E67
:100CE000E66EE66AA3D8E552E5520BD9020EF3CFC1
:100CF000DBFF030EF4CFDBFF04D9040EF3CFDBFFE1
:100D0000050EF4CFDBFF040EDBCF18F0050EDBCFB2
:100D100019F018C019F0186A020EDB501824146E6E
:100D2000030EDB501920156E166A176A15AE02D035
:100D300016681768060E14C0DBFF070E15C0DBFF30
:100D4000080E16C0DBFF090E17C0DBFF060EDBCF57
:100D500018F0070EDBCF19F0080EDBCF1AF0090EE2
:100D6000DBCF1BF018C004F019C005F01AC006F064
:100D70001BC007F007EC12F005C014F006C015F018
:100D800007C016F008C017F00A6A0B6A800E0C6ED6
:100D9000410E0D6E14C005F015C006F016C007F028
:100DA00017C008F020EC12F00A0E05C0DBFF0B0E96
:100DB00006C0DBFF0C0E07C0DBFF0D0E08C0DBFF1B
:100DC000C80EE66EE66A38DDE552E5520A0EDBCF64
:100DD00014F00B0EDBCF15F00C0EDBCF16F00D0E62
:100DE000DBCF17F014C004F015C005F016C006F0F4
:100DF00017C007F00E0EE15C03E200D0E16AE55295
:100E0000E16EE552E7CFD9FF1200926A8096010E9B
:100E1000E66EE66A11DDE552E552080E926E010EAD
:100E2000E66EE66A09DDE552E5521200D9CFE6FF2B
:100E3000E1CFD9FF040EE126020EDB6A030EDB6A66
:100E4000020EDBCF14F0030EDBCF15F0D890155057
:100E500004E6080E145C000E155849E2926A80966A
:100E6000020EE66E06EC19F0E552010EE76EFD0E7D
:100E7000DBCF14F0FE0EDBCF15F0E7501416156A29
:100E800014C0DEFF15C0DDFFD9CFE9FFDACFEAFFDE
:100E9000010EEE1801E1ED5001E18086D9CFE9FFA6
:100EA000DACFEAFFEE50ED1001E180963C0EE66EDF
:100EB00006EC19F0E552080E926E020EE66E06EC94
:100EC00019F0E552FD0EDBCF14F0FE0EDBCF15F06E
:100ED000D89015321432FD0E14C0DBFFFE0E15C083
:100EE000DBFF020EDB2A030E01E3DB2AA9D7040E87
:100EF000E15C02E2E16AE552E16EE552E7CFD9FF3B
:100F00001200D9CFE6FFE1CFD9FF040EE126DE6A59
:100F1000DD6ADECF14F0DDCF15F0D890155004E671
:100F2000080E145C000E15584BE2926A8096020E71
:100F3000E66E06EC19F0E552080E926EE66E06ECCF
:100F400019F0E552020EDBCF14F0030EDBCF15F0E3
:100F5000D89015321432020E14C0DBFF030E15C0F8
:100F6000DBFF80A610D0800EE76E020EDBCF14F000
:100F7000030EDBCF15F0E7501412020E14C0DBFF96
:100F8000030E15C0DBFF80B611D07F0EE76E020E98
:100F9000DBCF14F0030EDBCF15F0E7501416156A03
:100FA000020E14C0DBFF030E15C0DBFF780EE66EE9
:100FB00006EC19F0E552DF2A010E01E3DB2AA9D77E
:100FC000020EDBCF14F0030EDBCF15F014C0F3FFDD
:100FD00015C0F4FF040EE15C03E200D0E16AE552C3
:100FE000E16EE552E7CFD9FF1200DACFE4FFE2CF9E
:100FF000DAFFE65202011507000E165BD890165173
:10100000000A08E6000E135D000E1459010E155972
:10101000000E165909E21B0E1427B70E1523000EF9
:1010200016230001802B812300013C0E801901E171
:10103000815119E18C2B000E8D23806B816B3C0E4E
:101040008C1901E18D510FE18A2B000E8B238C6BE3
:101050008D6B180E8A1901E18B5105E1882B000E6A
:1010600089238A6B8B6BF294E552E5CFDAFF11008E
:1010700028DC80A809D880AA92D882A036D982A27A
:101080002DDA9AD9FFD712001CDC80DCA4DC010E1B
:1010900000019F259F6F000EA021A06F9D6B9E6B8E
:1010A000100E9EAF02D0D89003D09D5D000E9E59C9
:1010B0001AE29D519F25F66E9E51A021F76EB20E49
:1010C000F626280EF7220800F550E66E1B0E9D2529
:1010D000E96E020E9E21EA6EE552E750EF6E9D2BFF
:1010E000000E9E23DDD7E66AE66A7FDCE552E55214
:1010F00000019D6B9E6B080E9EAF02D0D89003D06E
:101100009D5D000E9E590FE21B0E9D25E96E020E9D
:101110009E21EA6EEF50E66E9CDCE55200019D2BAD
:10112000000E9E23E8D7E66A010EE66E5EDCE5520D
:10113000E552080E00019D6F9E6B100E9EAF02D00F
:10114000D89003D09D5D000E9E590FE21B0E9D2589
:10115000E96E020E9E21EA6EEF50E66E7ADCE552F1
:1011600000019D2B000E9E23E8D75E0EE66E010E59
:10117000E66E1CEC04F0E552E552100E0001F76A31
:101180009F25F66EA051F722B20EF626280EF72202
:101190000800F55002E19F6BA06B79D7120061EC5B
:1011A00004F0C6EC04F017DCA10EE66E000EE66E4D
:1011B00061DCE552E5526ADD04C02FF205C030F271
:1011C00006C031F207C032F22FC205F030C206F07D
:1011D00031C207F032C208F077EC13F006C033F2E8
:1011E00007C034F233C206F034C207F0F2EC11F05B
:1011F00005C018F006C019F007C01AF008C01BF0AF
:1012000018C00AF019C00BF01AC00CF01BC00DF08A
:101210002FC205F030C206F031C207F032C208F02A
:10122000E0EC12F005C014F006C015F007C016F08F
:1012300008C017F00A6A0B6A200E0C6E410E0D6E84
:1012400014C005F015C006F016C007F017C008F06E
:1012500073EC12F077EC13F006C035F207C036F2EB
:1012600035C2E6FF36C2E6FF33C2E6FF34C2E6FF10
:10127000380E146E320E156E166A14C0E6FF15C0D5
:10128000E6FF16C0E6FF370EE66E020EE66E26ECAF
:1012900017F0176E090EE15E1750E66A010EE66E52
:1012A000F5EC04F0E552E552370EE66E020EE66EFE
:1012B0003AEC05F0E552E552200EE66E29EC05F019
:1012C000E552D60EE66E29EC05F0E552430EE66EC9
:1012D00029EC05F0E552200EE66E030EE66E1CECDE
:1012E00004F0E552E55267D7120061EC04F0C6EC59
:1012F00004F0EBEC04F0E66AE66AF5EC04F0E55283
:10130000E5528E0EE66E000EE66E3AEC05F0E55202
:10131000E5523E0EE66E29EC05F0E552E66A010E56
:10132000E66EF5EC04F0E552E55234DC0A0EE66EAA
:10133000020EE66EB1EC16F0E552E552F3CF17F26D
:10134000F4CF18F20201196B1A6B18AF02D01969A9
:101350001A69500E171906E10D0E181903E11951FB
:1013600001E11A5115E1EBEC04F0950EE66E000E6A
:10137000E66E3AEC05F0E552E5528080D00EE66E5E
:10138000070EE66E1CEC04F0E552E552809012D098
:10139000EBEC04F09A0EE66E000EE66E3AEC05F009
:1013A000E552E552E80EE66E030EE66E1CEC04F024
:1013B000E552E5529ED7120061EC04F0C6EC04F051
:1013C000EBEC04F0010E00019F259F6F000EA021A1
:1013D000A06F9D6B9E6B100E9EAF02D0D89003D075
:1013E0009D5D000E9E591AE29D519F25F66E9E51FD
:1013F000A021F76E0A0EF6262B0EF7220800F550F4
:10140000E66E1B0E9D25E96E020E9E21EA6EE552E8
:10141000E750EF6E9D2B000E9E23DDD7E66AE66A4D
:10142000F5EC04F0E552E55200019D6B9E6B080E51
:101430009EAF02D0D89003D09D5D000E9E5910E261
:101440001B0E9D25E96E020E9E21EA6EEF50E66EA0
:1014500029EC05F0E55200019D2B000E9E23E7D7F5
:10146000E66A010EE66EF5EC04F0E552E552080E70
:1014700000019D6F9E6B100E9EAF02D0D89003D0DE
:101480009D5D000E9E5910E21B0E9D25E96E020E19
:101490009E21EA6EEF50E66E29EC05F0E552000160
:1014A0009D2B000E9E23E7D7130EE66E010EE66E0F
:1014B0001CEC04F0E552E552100E0001F76A9F257E
:1014C000F66EA051F7220A0EF6262B0EF722080020
:1014D000F55002E19F6BA06B75D7120061EC04F030
:1014E000816AF6D80201136B1B0E146FB70E156FCD
:1014F000166B9F0EE66E9CEC18F0E552F28E0ED83D
:1015000000018251801902E18351811905E080C0F8
:1015100082F081C083F052D8F3D71200D9CFE6FF12
:10152000E1CFD9FF100EE126D9CFE9FFDACFEAFFEC
:10153000480EEE6E4F0EEE6E520EEE6E410EEE6ED9
:101540003A0EEE6EEE6AD950060FE96EDACFEAFF78
:10155000300EEE6EEE6E3A0EEE6E300EEE6EEE6EFB
:101560003A0EEE6E300EEE6EEE6EEE6AEE6AC6EC7F
:1015700004F0EBEC04F0D9CFE6FFDACFE6FF3AEC6B
:1015800005F0E552E552E66A010EE66EF5EC04F070
:10159000E552E552D950060FE66E000EDA20E66EEF
:1015A0003AEC05F0E552E552100EE15C02E2E16A28
:1015B000E552E16EE552E7CFD9FF1200D9CFE6FF41
:1015C000E1CFD9FF0A0EE126E66A010EE66EF5ECE0
:1015D00004F0E552E5528AC0E6FF8BC0E6FF330E09
:1015E000146E320E156E166A14C0E6FF15C0E6FFC3
:1015F00016C0E6FFD9CFE6FFDACFE6FF26EC17F0FC
:10160000176E070EE15E1750D9CFE6FFDACFE6FF7F
:101610003AEC05F0E552E552030EE66E010EE66E79
:10162000F5EC04F0E552E5528CC0E6FF8DC0E6FF14
:10163000330E146E320E156E166A14C0E6FF15C016
:10164000E6FF16C0E6FFD9CFE6FFDACFE6FF26ECCD
:1016500017F0176E070EE15E1750D9CFE6FFDACF0D
:10166000E6FF3AEC05F0E552E552060EE66E010E95
:10167000E66EF5EC04F0E552E55280C0E6FF81C06D
:10168000E6FF330E146E320E156E166A14C0E6FFB6
:1016900015C0E6FF16C0E6FFD9CFE6FFDACFE6FFBA
:1016A00026EC17F0176E070EE15E1750D9CFE6FF54
:1016B000DACFE6FF3AEC05F0E552E5520A0EE15CBE
:1016C00002E2E16AE552E16EE552E7CFD9FF12008E
:1016D000D9CFE6FFE1CFD9FF080EE126D950030F9D
:1016E000E96EDACFEAFF530EEE6E450EEE6E540E43
:1016F000EE6E3E0EEE6EEE6AC6EC04F0EBEC04F01D
:10170000D950030FE66E000EDA20E66E3AEC05F0D3
:10171000E552E552E66A010EE66EF5EC04F0E5529C
:10172000E552CAEC05F0E66A010EE66EF5EC04F04F
:10173000E552E552F4EC05F00AC2DFFF010E0BC2E0
:10174000DBFF020EDB6AD9CFE6FFDACFE6FFB1ECB2
:1017500016F0E552E552F3CF8AF0F4CF8BF00CC2CD
:10176000DFFF010E0DC2DBFF020EDB6AD9CFE6FF01
:10177000DACFE6FFB1EC16F0E552E552F3CF8CF08C
:10178000F4CF8DF00EC2DFFF010E0FC2DBFF020EA1
:10179000DB6AD9CFE6FFDACFE6FFB1EC16F0E5520F
:1017A000E552F3CF80F0F4CF81F0080EE15C02E265
:0E17B000E16AE552E16EE552E7CFD9FF120083
:0217BE001BEC22
:1017C00011F0FB0EDBCFF3FFDB06F35000090AE05C
:1017D00069EC11F0FA0ED4EC11F0F3E1151CF1E113
:1017E000010E01D0000E4AEF11F01BEC11F03B0E80
:1017F000E12402E3E168E652E16E010EDB6A020ECB
:10180000DB6AF90EDBCFF6FFFA0EDBCFF7FFFB0E3C
:10181000DBCFF8FF0800F550DF6EDF5002E16EEF1E
:1018200010F0250EDF5C02E061EF10F0030EDB6AC2
:10183000040EDB6A050EDB6A060EDB6A070EDB6A46
:1018400083EC10F02D0EDF5C0CE02B0EDF5C09E06A
:10185000200EDF5C06E0230EDF5C03E0300EDF5C71
:101860001AE1DF50300A14E0130A0FE0030A0AE01D
:101870000B0A05E0060AE4E1030EDB80E1D7030E64
:10188000DB82DED7030EDB84DBD7030EDB86D8D703
:10189000030EDB88D5D72A0EDF5C1BE17FEC10F04E
:1018A000CDEC10F010E0030EDB8006680768130E25
:1018B000DBCF0BF0140EDBCF0CF02CEC14F0040E8D
:1018C00004C0DBFF03D0130EB6EC10F083EC10F075
:1018D0000BD0090EDB6A24EC11F003E098EC11F058
:1018E000FAD7090EB6EC10F0030EDBB0DB982E0E23
:1018F000DF5C1BE183EC10F02A0EDF5C0BE17FEC78
:1019000010F0CDEC10F003E1130E08EC11F083ECB5
:1019100010F00BD0090EDB6A24EC11F003E098EC18
:1019200011F0FAD7090E08EC11F0680EDF5C07E140
:1019300083EC10F0680EDF5C1DE1030E18D0740E0E
:10194000DF5C17E07A0EDF5C14E0480EDF5C06E037
:10195000540EDF5C03E05A0EDF5C02E1020E07D09A
:101960006C0EDF5C03E06A0EDF5C04E1010E5BECF1
:1019700011F0C9DBDF506E0A01E17FD31E0A01E1DD
:1019800092D1200A01E18FD13F0A01E149D11A0A1F
:1019900001E146D10D0A01E143D1200A01E140D124
:1019A0003A0A01E13DD1200A01E13AD1260A01E1DA
:1019B00035D10D0A01E132D11A0A01E1D9D0200A4C
:1019C0004AE0300A1FE0460A0EE0250A01E083D310
:1019D000D950F90FE96EFF0EDA20EA6E010EEE5EC5
:1019E000000EEE5AEE5A69EC11F0250EE66E95DB0C
:1019F00003E1151C01E169D365EC11F001E26BD341
:101A0000DB2A69D3080EDB6A040EDB50010806E20C
:101A1000040EDB042DEC11F0DB508BDB080EDB50E9
:101A200009E0030EDB50010B05E172DB01E04DD351
:101A3000080EDB6A64DBEFCFDFFFDDEC11F003E1C2
:101A4000151C01E142D365EC11F001E3DB2A60DBF8
:101A500001E141D33AD3070EDB5002080FE1A9ECB4
:101A600011F0030E70EC11F00E0EEECFDBFF0F0E37
:101A7000EECFDBFF100EEECFDBFF20D0F70EDBCF7B
:101A800017F0F80EDBCF18F0020E175E000E185A92
:101A9000F70E17C0DBFFF80E18C0DBFF17C0E9FF19
:101AA00018C0EAFF60EC11F0166A0E0E14C0DBFFDE
:101AB0000F0E15C0DBFF100E16C0DBFF0E0EDBCFC6
:101AC000E6FF0F0EDBCFE6FF100EDBCFE6FF53EC99
:101AD00018F0E552E552E552130E05C0DBFF140E77
:101AE00006C0DBFF060EDB5005E0130EA4EC11F080
:101AF00001E26ADBC8EC11F002E2130E37DB8BEC7B
:101B000011F006E0040EA4EC11F002E2050E2EDB4B
:101B1000030EDBB005D0FCDA01E0D7D2080EDB6A99
:101B2000090EDB6A0E0EDBCFF6FF0F0EDBCFF7FFE1
:101B3000100EDBCFF8FF0800F550DF6EDF5014E029
:101B4000CEEC11F011E2DDEC11F003E1151C01E126
:101B5000BCD2BBDB01E3DB2A090EDB2AD9500E0F16
:101B6000E96E000ECBDBE7D7D3DA01E1B4D2ADD218
:101B7000C6DA110EEECFDBFF120EEDCFDBFF110E3A
:101B8000DBCFE6FF120EDBCFE6FF45EC18F0E552A7
:101B9000E552130EF3CFDBFF140EF4CFDBFF060E7E
:101BA000DB5004E0130ED0DB01E20EDBC8EC11F0D9
:101BB00002E2130EDBDAAFDB05E0040EC5DB02E266
:101BC000050ED4DA030EDBB005D0A2DA01E07DD237
:101BD000080EDB6A090EDB6A110EDBCFE9FF120E7D
:101BE000DBCFEAFFEFCFDFFFDF5014E0D7DB12E2FD
:101BF000E4DB03E1151C01E168D267DB01E3DB2ACA
:101C0000090EDB2A110EDB2ADBCFE9FF120EE8E317
:101C1000DB2AE6D77DDA01E15ED257D2030EDB8EF6
:101C2000070EDB0410E195DB040E5ADB0A0EEECF43
:101C3000DBFF0B0EEECFDBFF0C0EEECFDBFF0D0E4E
:101C4000EECFDBFF6CD0070EDB5003082CE1030E58
:101C5000DBAE0DD0B2DA020E76DAEFCF14F0156AF1
:101C6000166A176A14AE39D01568166835D0F70EA3
:101C7000DBCF15F0F80EDBCF16F0020E155E000E6E
:101C8000165AF70E15C0DBFFF80E16C0DBFF15C0A5
:101C9000E9FF16C0EAFFEFCF14F00A0E14C0DBFF15
:101CA0000B0EDB6A38D0070EDB50020809E1030E89
:101CB000DBAE04D059DB16AE10D00ED055DB0DD004
:101CC000030EDBAE12D079DA020E3DDAF9DA166ACB
:101CD000176A15AE02D016681768E2DA0C0E16C045
:101CE000DBFF0D0E17C0DBFF1AD0F70EDBCF16F0AF
:101CF000F80EDBCF17F0020E165E000E175AF70E25
:101D000016C0DBFFF80E17C0DBFF16C0E9FF17C0D7
:101D1000EAFFD6DAC5DA0C0EDB6A0D0EDB6A060EB8
:101D2000DB5005E1010EF36E050EF3CFDBFF150E60
:101D3000DB6A160EDB6AD950370F146E000EDA20FC
:101D4000156E390E14C0DBFF3A0E15C0DBFF380EDE
:101D5000DB6A080EDB6A0A0EAEDADF50780A12E0A0
:101D6000200A10E0280A0CE0200A0AE03F0A06E0F8
:101D70000D0A02E0200A08E1020E05D0080E03D089
:101D8000080EDF26100E97DA030EDBBE02D0DB92C0
:101D9000DB94DB50800B24E08ADAD890030EEB5002
:101DA000000A08E6000EEE5C000EEE58000EEE583B
:101DB000000EEE5815E213DA09680A680B680C6821
:101DC0000DEC18F00A0E00C0DBFF0B0E01C0DBFFAC
:101DD0000C0E02C0DBFF0D0E03C0DBFF2D0E08D082
:101DE000030EDBA202D02B0E03D0DBA408D0200E02
:101DF000F36E170EF3CFDBFF150EDB2A02D0170EA2
:101E0000DB6A050EDB5003E1B7D901E189D0220E70
:101E1000146E320E156E000E166E070EDBCF17F025
:101E2000186A196A1A6A17C009F018C00AF019C0AE
:101E30000BF01AC00CF0D3D978EC18F01450002431
:101E4000F36E15500120F46E16500220F86EF4CF98
:101E5000F7FFF3CFF6FF0800090EF5CFDBFF580EB2
:101E6000DF5C0FE1610EF36E090E7BD90AE3200EF1
:101E7000146E090EDBCFE7FF1450E75E090EE7CFC3
:101E8000DBFF070EDBCF14F0156A166A176A0FDA4C
:101E900014C009F015C00AF016C00BF017C00CF002
:101EA000EECF04F0EECF05F0EECF06F0EFCF07F067
:101EB00078EC18F007C0EDFF06C0EDFF05C0EDFFA0
:101EC00004C0EFFF390EDBCFE9FFDB063A0EDBCFB4
:101ED000EAFF01E2DB06090EDBCFEFFF150EDB2A7E
:101EE0004BD995E1030EDBA61DD06F0EDF5C06E13A
:101EF000C1D918E3150EDB285BDA14D0780EDF5C4D
:101F000009E0580EDF5C06E0620EDF5C03E0420E83
:101F1000DF5C08E1020EF36E160EF3CFDBFF02D09A
:101F2000150EDB6A030EDB50100B0EE0040EDBCF48
:101F300014F0050EDB50D880145406E2060EDB5078
:101F400003E1040EDB5034DA95D90AE2050EDBCF4B
:101F5000E7FF150EDB50E75E050EE7CFDBFF02D093
:101F6000050EDB6A040EDBCF14F0160E45D9D880BF
:101F7000145414E2160EDBCFE6FF150EDBCFE6FF9E
:101F8000040EDBCFE6FF050EDB50E552E75CE552C1
:101F9000D880E754E552D880E7545FD9030EDB5070
:101FA000010B0BE1080EDB5008E0B2D801E08DD048
:101FB000080EDB50BED8080EDB6A170EDB5007E0B8
:101FC00088D9170EF1D903E1151C01E17ED0160E58
:101FD000DB5016E07ED9300EE66E9FD802E1151C6C
:101FE00074E077D9DFCFE6FFCBEC17F0E552E5528E
:101FF000E552F4CF15F00001F31C02E1151C65E079
:10200000050EDBCF14F0160EDB50D880145409E215
:10201000050EDBCFE7FF160EDB50E75E050EE7CFC0
:10202000DBFF300EE66E050ECBD94FE1390EDB2A11
:10203000DBCFE9FF3A0E01E3DB2ADBCFEAFF090E33
:10204000EFCFDBFFDB500EE044D9090EADD902E142
:10205000151C3BE0390EDB2ADBCFE9FF3A0EEDE33E
:10206000DB2AEBD755D831E1160EDBCFE6FF080EA1
:10207000C3D8E552E7245DD82ED0070EDB50030A03
:102080001CE0010A14E0030A07E07BD9DBCFEEFF76
:10209000020EDBCFEDFF1FD0F5D8196A17AE02D0C4
:1020A000186819682CD8BCD819C0EEFF14D0EAD82B
:1020B00017BE186824D8B4D80ED063D9DBCFEFFF91
:1020C0000AD07BD905E1151C03E1F368F46810D050
:1020D000FCD801E3DB2A79D90AEF0CF0010EDBCF43
:1020E00014F0020EDBCF15F014C0F3FF15C0F4FF9F
:1020F0003B0EE15C02E2E16AE552E16ECBD029D908
:10210000020E70EF11F061D90800F550DF6E120079
:10211000200EE66E080EE0EF11F0CBEC17F0E55262
:10212000E552E552F3CF14F0F4CF15F00001F31CA3
:102130001200146E156AD950010F4DD91450EE26B5
:102140001550ED221200185E000E195AF70E18C035
:10215000DBFFF80E19C0DBFF18C0E9FF19C0EAFF6A
:102160001200DBCFF4FFF350F45C1200DB50E76E9B
:10217000040EE7CFDBFF12000A0EDBCF14F00B0ECC
:10218000DBCF15F00C0EDBCF16F00D0EDBCF17F00A
:1021900014501510161017101200130EEECFDBFF9F
:1021A000140EEDCFDBFF130EDBCF14F0140EDBCFDC
:1021B00015F00001800E15141200F70EDBCF18F099
:1021C000F80EDBCF19F01200050EDB50E66ED95089
:1021D000130F01D9E552E750EE6EED6A12000A0EB8
:1021E000DBCF04F00B0EDBCF05F00C0EDBCF06F0DF
:1021F0000D0EDBCF07F01200DBCFE6FF150EDBCFB5
:10220000E6FF050EDB50E552E724E552E724120015
:10221000DB50CED8010EF36E060EF3CFDBFF1200BB
:10222000EE50EFCFEAFFE96E16C0EEFF17C0EEFFEB
:1022300018C0EEFF1200D9CFE6FFDACFE6FFE1CFFC
:10224000D9FFE2CFDAFF1200DFCFE6FFE66AB8EC93
:1022500018F0E552E552F3501200E76E080EE7CF92
:10226000DBFF1200EECF14F0EECF15F0EFCF16F03B
:10227000176A1200050EDBCF14F0150EDB50D88064
:1022800014541200010EDBCF16F0020EDBCF17F054
:10229000186A1200E552E5CFDAFFE7CFD9FF120046
:1022A0000A0E14C0DBFF0B0E15C0DBFF1200D95065
:1022B0000A0FEBEF11F0F36E070EF3CFDBFF120006
:1022C000EECF14F0EFCF15F01200010EDB2A020E54
:1022D0001200FC0EDBCFE6FFFD0EDBCFE6FF1200A7
:1022E000145E000E155AF70E14C0DBFFF80E15C071
:1022F000DBFF14C0E9FF15C0EAFF1200DA20EA6E26
:10230000EF2AEECFF6FF000EEF22EECFF7FFEF221F
:10231000EECFF8FF1200040EDBCFE6FF130EDB500A
:10232000E552E75C9ADFDB5004DF060EDB5012005B
:10233000090EDB500A0DF350DF24D00FE76E090EB3
:10234000E7CFDBFF83EF10F0DB50F36E050EB1EF4C
:1023500010F0F70EDBCF14F0F80EDBCF15F0120003
:10236000DFCFE6FF8DEF10F028DF030EECDE32EF5B
:1023700011F0DFEC0BF0E552E552E552E5520009B1
:102380001200BDDEEE50EFCFEAFFE96E010E120043
:10239000130EDB50F36E040EB1EF10F0040EDB50A1
:1023A000F36E090EB1EF10F0DBCFE6FF8DEF10F00A
:1023B000E76E050EE7CFDBFF12008BDFB0EF11F009
:1023C000DBCFE6FF86DFB9EF11F0D950F90FE96EE8
:1023D000FF0E7EEF11F0E96E000EDA20EA6E1200B9
:1023E0000F9E08D00F9E07AE05D0066C071EE86A48
:1023F00007220F8E07C001F006C000F0136A126AB0
:102400008E0E026E036AC2EF13F00F9E0CD00F9E69
:1024100007AE09D0046C051E061E071EE86A0522D9
:10242000062207220F8E07C001F006C000F005C08B
:1024300013F004C012F09E0E026E036AC2EF13F096
:102440000F6AFEEC13F016EC14F00FB6A6EF13F0C3
:102450000FA205D00FBAA6EF13F0ADEF13F00FBA2D
:10246000B9EF13F00FA005D00FB8A6EF13F0B9EF36
:1024700013F00FB8ADEF13F0036A7F0E0824026E5D
:10248000E86A03220D50025EE86A035A1A0E106EC3
:10249000086A126A136A006A016A0A50055E0B50E4
:1024A000065A0C50075A000E085A09E70A5005262A
:1024B0000B5006220C500722000E082201D0128A6F
:1024C000D8900536063607360836D89012361336B9
:1024D00000360136102EE1D7075006100510D8A49B
:1024E000128AC2EF13F00F6AFEEC13F016EC14F030
:1024F0000FB6A6EF13F00FA205D00FB8A6EF13F09A
:10250000ADEF13F00FAA05D00FB0A6EF13F0ADEFAB
:1025100013F00FB002D00FA802D0B9EF13F0036A86
:102520000D500824026EE86A03227E0E025EE86AFD
:10253000035A126A136A006A016A0C500702F4CF48
:1025400001F0F3CF00F00B500702F3501326F450C4
:102550000022000E01220C500602F3501326F45004
:102560000022000E01220A500702F3501226F450F6
:102570001322000E002201220B500602F3501226F5
:10258000F4501322000E002201220C500502F350D9
:102590001226F4501322000E002201220A500602D5
:1025A000F4501226000E1322002201220B500502C5
:1025B000F4501226000E132200220122C2EF13F063
:1025C0000D7E0F6AFEEC13F016EC14F00FB6A6EFBA
:1025D00013F00FA20AD00FAA03D00FBEA6EF13F07C
:1025E0000FA4B2EF13F0AFEF13F00FAA05D00FACAA
:1025F000B2EF13F0AFEF13F00FA00AD00FA808D07E
:102600000FBE04D00FA402D0BBEF13F0BFEF13F046
:10261000126A036A0D50085C116E10E305C013F0D6
:1026200006C000F007C001F008C010F00AC005F0B5
:102630000BC006F00CC007F00F3A09D00AC013F027
:102640000BC000F00CC001F00DC010F0116C0F9E1B
:102650000FBC0F8E10C002F00FB0EEEF13F01A0E89
:102660001160EEEF13F0026A086A0FA408D0056C3F
:10267000061E071E081EE86A0622072208220FAC63
:1026800008D0136C001E011E021EE86A00220122FF
:102690000222046A115207E008340732063205327A
:1026A0000432112EF9D70550132606500022075088
:1026B00001220850022204C012F00F9E02AE0BD07D
:1026C000126C131E001E011E021EE86A1322002255
:1026D000012202220F8E02A006D0D88001320032E1
:1026E00013321232102A10C002F0C2EF13F00F6A38
:1026F000FEEC13F00FB681EF13F00FA20ED00FB463
:1027000005D07F0E076EFF0E066E1FD0800E076E7F
:10271000066A1BD0076A066A18D00FB0FBD78F0E67
:102720000860EDD77E0E0864F5D78E0E085C05E0D4
:10273000D89007320632082AF8D70FA406D0066CC4
:10274000071EE86A072207AEE5D712007F0E086E63
:10275000FF0E076E066E056E12007F0E0FBEFF0E97
:10276000086E02D07F0E086E800E076E066A056A3C
:10277000F3D70FAE04D0800E086E076AF7D7086A49
:10278000076AF4D70150001013101210F8E003BECE
:10279000F0D701BE0CD002500310EBE0D8901236F7
:1027A0001336003601360206D8A00306F2D70350CE
:1027B000D4E10228D2E012AE11D07F0E121402E151
:1027C00013A00CD0132AE86A0022012207E3D88064
:1027D000013200321332022A0228BFE00250C9E05F
:1027E00013C005F000C006F00134076E0230086E19
:1027F0000732089E0FBE088EACEF13F0073608367E
:1028000002E30F840F7E06E10F80086A076A066AFA
:10281000056A1200082803E0D88007321200D89019
:10282000073202E10F8212000F8612000C360D36BD
:1028300002E30F8C0F7E06E10F880D6A0C6A0B6AAB
:102840000A6A12000D2803E0D8800C321200D890DA
:102850000C32EAE10F8A120007C013F006C012F032
:1028600006500B02F4CF05F0F3CF04F007500C0232
:10287000F4CF07F0F3CF06F00B02F3500526F45027
:102880000622E86A072212500C02F3500526F45083
:102890000622E86A07220CAE52EF14F01250065ED0
:1028A0001350075A13AE000C0B50065E0C50075A1B
:0228B000000C1A
:0E28B2002E2E2E2E2E2E2E2E2E2E2E2E2E2E94
:1028C0002E2E53495354454D4120424F4C542031F4
:1028D0003846323535302E2E3230204D485A2E2E85
:1028E00033324B204D454D4F52494120464C4153C8
:1028F000482E2E324B204D454D4F524941205241DA
:102900004D2E2E3235362042595445532044452011
:10291000454550524F4D2E2E53454E534F52204455
:10292000452054454D504552415455524120445341
:1029300031384232302E2E52454C455641444F528A
:102940002044452031323720562E2061203120414D
:102950004D502E2E38204C4544532E2E34204D49B8
:1029600043524F53574954434845532E2E505545D3
:1029700052544F2055534220434F4E2050524F4700
:1029800052414D41444F5220494E544547524144D3
:102990004F2E2E50554552544F2053455249414CCD
:1029A0002052532D3233322E2E50554552544F5310
:1029B0002050415241204C43442059205445434C1F
:1029C00041444F2E2E534F465457415245204445C3
:1029D000204445534152524F4C4C4F2050524F4689
:1029E0004553494F4E414C2C20494E434C55594577
:1029F000204D504C4142204944452E2E2E434F4DF0
:102A000050494C41444F52204331382E2E2E534FC3
:102A10004654574152452044452050524F47524159
:102A20004D4143494F4E2E2E2E2E2E2E2E2E2E2E23
:102A30002E2E2E2E2E0000000000000000000000B0
:102A40000000000000000000000000000000000086
:102A50000000000000000000000000000000000076
:102A60000000000000000000000000000000000066
:102A70000000000000000000000000000000000056
:102A80000000000000000000000000000000000046
:102A90000000000000000000000000000000000036
:102AA0000000000000000000000000000000000026
:102AB0000000000000000000000000000000000016
:102AC0000000000000000000000000000000000006
:102AD00000000000000000000000000000000000F6
:102AE00000000000000000000000000000000000E6
:102AF00000000000000000000000000000000000D6
:102B0000000000000000000000002E2E2E2E2E2EB1
:102B10002E2E2E2E2E2E2E2E2E2E50554E544F2033
:102B2000464C4F54414E544520532E412E2E2E5389
:102B3000495354454D4120424F4C54203138463280
:102B40003535302E2E50524F4752414D412044458D
:102B50002044454D4F5354524143494F4E20434F1B
:102B60004E20342041504C49434143494F4E455338
:102B70003A205357313D4F4E203E3E20204D554583
:102B800053545241204C41532043415241435445F8
:102B900052495354494341532044454C204D4F44DE
:102BA000554C4F20424F4C54203138463235353049
:102BB0002E2E5357323D4F4E203E3E2041504C4921
:102BC000434143494F4E2053454E534F52204445B5
:102BD0002054454D50455241545552412E2E535785
:102BE000333D4F4E203E3E2041504C4943414349E6
:102BF0004F4E20434841504120454C454354524F8D
:102C00004E4943412C20434C4156453D33343038E6
:102C100020444553444520454C205445434C4144B1
:102C20004F2048455841444543494D414C20284F89
:102C30005052494D412027462720414C2046494EBD
:102C4000414C292E2E5357343D4F4E203E3E2052AC
:102C5000454C4F4A204445205449454D504F205241
:102C600045414C2C494E54524F44555A43412044FF
:102C70004553444520454C205445434C41444F2046
:102C80004C4120484F52412C4D494E55544F532CE6
:102C9000534547554E444F5320434F4E2036204412
:102CA000494749544F5320434F4E53454355544988
:102CB000564F5320592027462720414C2046494E45
:102CC000414C2E2E44415220524553455420414CF4
:102CD000204D4F44554C4F205041524120494E49C0
:102CE0004349415220434144412041504C494341D2
:102CF00043494F4E2E2E2E2E2E2E2E2E2E2E2E2E83
:102D00002E2E2E2E0000000000000000000000000B
:102D100000000000000000000000000000000000B3
:102D200000000000000000000000000000000000A3
:102D30000000000000000000000000000000000093
:102D40000000000000000000000000000000000083
:102D50000000000000000000000000000000000073
:022D6000000071
:0E2D6200FF0EE3CFEAFFE552FF0EE3CFE9FFDD
:102D7000E552E66AE66AD9CFE6FFDACFE6FFFC0E57
:102D8000E124D96EFF0EE220DA6EE66AE66AE66AB0
:102D9000200EEF5C06E0090EEF5C03E0EF6603D067
:102DA0003FD0EE50F5D72D0EEF5C03E1FF0EE32A86
:102DB00003D02B0EEF5C01E1EE502F0EEF6424D018
:102DC0003A0EEF6021D0D890F90EE336FA0EE336D2
:102DD000FD0EDECFE3FFFE0EDDCFE3FFD890F90E50
:102DE000E336FA0EE336D890F90EE336FA0EE33600
:102DF000FD0EE350DE26FE0EE350DD22300EEE5CCB
:102E0000DE26000EDD22D9D7FF0EE3CFE8FFE85221
:102E100007E0F90EE31EE32AFA0ED8B4E306E31E38
:102E2000E552E552E552FF0EE3CFDAFFE552FF0E21
:102E3000E3CFD9FFE552E1CFE9FFE2CFEAFFED5260
:0C2E4000ED52EECFF3FFEFCFF4FF1200D5
:042E4C00D9CFE6FFF5
:102E5000DACFE6FFE1CFD9FFE2CFDAFFE652E65262
:102E6000E652E652D950F90F146EFF0EDA20156EB5
:102E7000020E14C0DBFF030E15C0DBFF020EDBCF1A
:102E8000E6FF030EDBCFE6FFF90EDBCFE6FFFA0E1F
:102E9000DBCFE6FFFB0EDBCFE6FFD950FC0FE66E83
:102EA000FF0EDA20E66EF5EC0BF0146E070EE15C17
:102EB00002E2E16AE552E16E1450F3CFDEFFF4CF97
:102EC000DDFFFC0EDBCFE9FFFD0EDBCFEAFFEF6A93
:102ED000DECF14F0DDCF15F014C0F3FF15C0F4FF02
:102EE000040EE15C02E2E16AE552E16EE552E5CFF3
:082EF000DAFFE7CFD9FF120061
:082EF8002A0EF66E080EF76EBB
:102F0000000EF86E00010900F550AD6F0900F55094
:102F1000AE6F03E1AD6701D03DD00900F550A86F59
:102F20000900F550A96F0900F550AA6F09000900C2
:102F3000F550E96E0900F550EA6E09000900090034
:102F4000F550AB6F0900F550AC6F09000900F6CFE2
:102F5000AFF0F7CFB0F0F8CFB1F0A8C0F6FFA9C03E
:102F6000F7FFAAC0F8FF0001AB5302E1AC5307E042
:102F70000900F550EE6EAB07F8E2AC07F9D7AFC029
:102F8000F6FFB0C0F7FFB1C0F8FF0001AD07000EBB
:062F9000AE5BBFD712008A
:0A2F9600D9CFE6FFDACFE6FFE1CF66
:102FA000D9FFE2CFDAFFFB0EDBCF14F0FC0EDBCF54
:102FB00015F00001800E15141AE1FB0EDBCFE9FFBE
:102FC000FC0EDBCFEAFFEECFF3FFEDCFF4FFEE2AEE
:102FD000000EEF22F3CFE9FFF4CFEAFFFD0EDBCFC7
:102FE000EFFFEF50156AF36E15C0F4FF10D0FB0E23
:102FF000DB50FE0806E1FD0EDBCFE6FFF8EC18F033
:1030000005D0FD0EDBCFE6FF20EC19F0E552E552CE
:0A301000E5CFDAFFE7CFD9FF120089
:06301A0004500902F3CF8F
:1030200000F0F4CF01F00A02F3500126000EF42064
:10303000026E04500B02F3500226000EF420036EC1
:1030400004500C02F350032605500902F3500126E8
:10305000F4500222000E032205500A02F350022609
:10306000F450032205500B02F350032606500902C8
:10307000F3500226F450032206500A02F3500326AE
:0A30800007500902F3500326120066
:06308A00FE0EE3CFE9FF9A
:10309000FF0EE3CFEAFFF36AF46AEE5203E0F34A6D
:1030A000F42AFBD71200FF0EE3CFF8FFE552FF0E24
:1030B000E3CFF7FFE552FF0EE3CFF6FFE552E66AF6
:1030C000E66AE66A0900F55209E0FD0EE32A05E129
:1030D000FE0EE32A02E1FF0EE32AF4D7FD0EE3CF52
:1030E00005F0FE0EE3CF06F0FF0EE3CF07F012006F
:1030F000036A026A016A006A200EE76ED8900436FD
:1031000005360636073600360136023603360950D4
:10311000005C0A5001580B5002580C50035809E348
:103120000950005E0A50015A0B50025A0C50035AC3
:08313000042AE72EE4D7120087
:08313800D9CFE6FFDACFE6FF74
:10314000E1CFD9FFE2CFDAFFFD0EDB507F0BD56E6A
:10315000D76AD66AF294FD0EDBAE02D0F28A01D0B5
:10316000F29AD58EE552E5CFDAFFE7CFD9FF12000C
:10317000F36AF46AFF0EE124E96EFF0EE220EA6EC4
:10318000ED6607D02F0EEF6404D03A0EEF6001D049
:04319000F32A12000C
:0C319400FF0EE3501C6E480E01D04C0EE4
:1031A000E76EE72EFED7E76AE72EFED71C2EF7D78D
:0431B0000000120009
:0C31B400000EF36E00EE00F0080E01D8D3
:1031C0001200EA6002D0EE6AFCD7F350E960120008
:0431D000EE6AFCD7D0
:0C31D40012EE40F022EE40F0F86A0F9C72
:1031E0007CEC17F021EC19F038EC08F0FBD712005A
:1031F000FF0EE350ACBA04D0AF6AAB8EAC8A949C9D
:0C320000ACA2FED7AD6EF36EF46A1200B3
:04320C00FF0EE3507E
:10321000E84E1200000000D000D000D0E82EFAD70F
:0232200012009A
:0E322200303132333435363738396162636407
:03323000656600D0
:0C32330025303275002533642E25640020
:0232400012007A
:02324200120078
:0C324400EEEDEBE7DEDDDBD7BEBDBBB777
:103250007E7D7B77303132333435363738394142F1
:10326000434445460000000000000000000000004C
:103270000000434C4156453A004F4B2121006E6FF0
:0C328000000000000054454D50453D008A
:00000001FF
